:100000000C9458000C9480000C9480000C94800098
:100010000C9480000C9480000C9480000C94800060
:100020000C9480000C9480000C9480000C94DA00F6
:100030000C9480000C9480000C9480000C94800040
:100040000C949A030C9480000C94BD020C94EF0263
:100050000C9480000C9480000C9480000C94800020
:100060000C9480000C948000000000080002010045
:100070000003040700000000000000000102040863
:100080001020408001020408102001020408102002
:10009000040404040404040402020202020203032E
:1000A0000303030300000000250028002B001F03AA
:1000B00011241FBECFEFD8E0DEBFCDBF11E0A0E01E
:1000C000B1E0E2E9F8E002C005900D92A031B1077D
:1000D000D9F721E0A0E1B1E001C01D92A73BB20732
:1000E000E1F710E0C0EBD0E004C02297FE010E94CF
:1000F0004304CE3AD107C9F70E948B030C944704FE
:100100000C94000080E480937C0080917C008062ED
:1001100080937C0080917A00887F80937A00809120
:100120007A00846080937A0080917A008064809362
:100130007A0080917A0084FFFCCF0895ECE7F0E02C
:100140009081987F90839081982B90830895F89464
:1001500010928000E1E8F0E0108210928500109289
:10016000840088E09DE390938900809388008081DB
:1001700088608083808185608083EFE6F0E0808105
:10018000826080837894089526E040E054E863E03C
:1001900070E081E191E00E945B020E94A7000E9452
:1001A000820080E00E949E00EAE7F0E080818064A7
:1001B000808308951F920F920FB60F9211242F93F0
:1001C0003F934F935F936F937F938F939F93AF93DF
:1001D000BF93EF93FF93609110018DE00E94420165
:1001E0008091100191E0892780931001FF91EF9198
:1001F000BF91AF919F918F917F916F915F914F913F
:100200003F912F910F900FBE0F901F9018958091E6
:100210007A0084FFFCCF9091790080917A0080640D
:1002200080937A009093C6008091C00085FFFCCF38
:100230000895833081F028F4813099F08230A1F064
:1002400008958730A9F08830B9F08430D1F48091D6
:1002500080008F7D03C0809180008F778093800025
:10026000089584B58F7702C084B58F7D84BD0895CD
:100270008091B0008F7703C08091B0008F7D809314
:10028000B00008950F931F93CF93DF931F92CDB7C4
:10029000DEB7282F30E0F901E859FF4F8491F901CA
:1002A000E458FF4F1491F901E057FF4F04910023E8
:1002B000C9F0882321F069830E9419016981E02F28
:1002C000F0E0EE0FFF1FEC55FF4FA591B4919FB7E3
:1002D000F8948C91611103C01095812301C0812B8A
:1002E0008C939FBF0F90DF91CF911F910F91089535
:1002F000FC01818D228D90E0805C9F4F821B9109D3
:100300008F7399270895FC01918D828D981731F094
:10031000828DE80FF11D858D90E008958FEF9FEF9E
:100320000895FC01918D828D981761F0828DDF0117
:10033000A80FB11D5D968C91928D9F5F9F73928FD8
:1003400090E008958FEF9FEF089585E193E0892B6A
:1003500049F080E090E0892B29F00E94150381117B
:100360000C9400000895FC01848DDF01A80FB11DDD
:10037000A35ABF4F2C91848D90E001968F739927DB
:10038000848FA689B7892C93A089B1898C918064C8
:100390008C93938D848D981306C00288F389E02D89
:1003A00080818F7D80830895CF93DF93EC01888DCA
:1003B0008823C9F0EA89FB89808185FD05C0A88969
:1003C000B9898C9186FD0FC00FB607FCF5CF8081EF
:1003D00085FFF2CFA889B9898C9185FFEDCFCE0139
:1003E0000E94B301E7CFDF91CF910895CF92DF92C2
:1003F000FF920F931F93CF93DF931F92CDB7DEB77A
:100400006C0181E0D60158968C9358975B969C912D
:100410005B975C968C915C97981307C05096ED9112
:10042000FC915197808185FD2EC0F601038D10E06F
:100430000F5F1F4F0F731127F02EF601848DF812F6
:1004400011C00FB607FCF9CFD6015096ED91FC9183
:100450005197808185FFF1CFC60169830E94B30166
:100460006981EBCF838DE80FF11DE35AFF4F608365
:10047000D6015B960C935B975296ED91FC91539746
:10048000808180620CC0D6015696ED91FC91579701
:1004900060835096ED91FC915197808180648083B8
:1004A00081E090E00F90DF91CF911F910F91FF902D
:1004B000DF90CF900895BF92CF92DF92EF92FF929C
:1004C000CF93DF93EC016A017B01B22EE889F989B1
:1004D00082E08083411581EE580761057105A1F026
:1004E00060E079E08DE390E0A70196010E941F048F
:1004F000215031094109510956954795379527955E
:10050000211580E1380798F0E889F989108260E8C0
:1005100074E88EE190E0A70196010E941F0421502B
:100520003109410951095695479537952795EC852D
:10053000FD853083EE85FF852083188EEC89FD894B
:10054000B082EA89FB89808180618083EA89FB89A6
:10055000808188608083EA89FB89808180688083CC
:10056000EA89FB8980818F7D8083DF91CF91FF9025
:10057000EF90DF90CF90BF9008951F920F920FB62B
:100580000F9211242F938F939F93EF93FF93E091FA
:100590002101F09122018081E0912701F091280151
:1005A00082FD12C0908180912A018F5F8F7320910C
:1005B0002B01821751F0E0912A01F0E0EF5EFE4F2F
:1005C000958F80932A0101C08081FF91EF919F91C7
:1005D0008F912F910F900FBE0F901F9018951F9223
:1005E0000F920FB60F9211242F933F934F935F9367
:1005F0006F937F938F939F93AF93BF93EF93FF93EB
:1006000081E191E00E94B301FF91EF91BF91AF9121
:100610009F918F917F916F915F914F913F912F911A
:100620000F900FBE0F901F90189581E191E00E94EE
:10063000780121E0892B09F420E0822F089510929F
:1006400014011092130188EE93E0A0E0B0E08093D3
:10065000150190931601A0931701B093180184E03F
:1006600091E0909312018093110185EC90E09093BA
:100670001E0180931D0184EC90E0909320018093F3
:100680001F0180EC90E0909322018093210181EC86
:1006900090E0909324018093230182EC90E090936A
:1006A00026018093250186EC90E0909328018093A9
:1006B000270110922A0110922B0110922C01109206
:1006C0002D010895CF92DF92EF92FF920F931F9327
:1006D000CF93DF937C016A01EB0100E010E00C1581
:1006E0001D0571F06991D701ED91FC910190F081A8
:1006F000E02DC7010995892B19F00F5F1F4FEFCF30
:10070000C801DF91CF911F910F91FF90EF90DF9083
:10071000CF90089508950E94E4030E948A030E94E6
:10072000C400C5EAD1E00E9407012097E1F30E94CE
:10073000A501F9CF1F920F920FB60F9211242F939C
:100740003F938F939F93AF93BF938091AF0190910D
:10075000B001A091B101B091B2013091AE0123E09E
:10076000230F2D3720F40196A11DB11D05C026E8E9
:10077000230F0296A11DB11D2093AE018093AF01FE
:100780009093B001A093B101B093B2018091B301F5
:100790009091B401A091B501B091B6010196A11D4F
:1007A000B11D8093B3019093B401A093B501B093B0
:1007B000B601BF91AF919F918F913F912F910F9073
:1007C0000FBE0F901F901895789484B5826084BDF9
:1007D00084B5816084BD85B5826085BD85B5816045
:1007E00085BDEEE6F0E0808181608083E1E8F0E0A5
:1007F0001082808182608083808181608083E0E8D4
:10080000F0E0808181608083E1EBF0E080818460B2
:100810008083E0EBF0E0808181608083EAE7F0E0B4
:100820008081846080838081826080838081816018
:1008300080838081806880831092C1000895A1E246
:100840001A2EAA1BBB1BFD010DC0AA1FBB1FEE1F4A
:10085000FF1FA217B307E407F50720F0A21BB30B95
:10086000E40BF50B661F771F881F991F1A9469F711
:1008700060957095809590959B01AC01BD01CF016D
:100880000895EE0FFF1F0590F491E02D0994F89460
:02089000FFCF98
:1008920000000000F6016203780191018301D40196
:107800000C94343C0C94513C0C94513C0C94513CE1
:107810000C94513C0C94513C0C94513C0C94513CB4
:107820000C94513C0C94513C0C94513C0C94513CA4
:107830000C94513C0C94513C0C94513C0C94513C94
:107840000C94513C0C94513C0C94513C0C94513C84
:107850000C94513C0C94513C0C94513C0C94513C74
:107860000C94513C0C94513C11241FBECFEFD8E036
:10787000DEBFCDBF11E0A0E0B1E0ECE9FFE702C060
:1078800005900D92A230B107D9F712E0A2E0B1E065
:1078900001C01D92AD30B107E1F70E942D3D0C945F
:1078A000CC3F0C94003C982F959595959595959582
:1078B000905D8F708A307CF0282F295A8091C0000B
:1078C00085FFFCCF9093C6008091C00085FFFCCF60
:1078D0002093C6000895282F205DF0CF982F809127
:1078E000C00085FFFCCF9093C6000895EF92FF92F1
:1078F0000F931F93EE24FF2487018091C00087FD22
:1079000017C00894E11CF11C011D111D81E4E8164B
:1079100082E4F8068FE0080780E0180770F3E09132
:107920000401F091050109958091C00087FFE9CF1E
:107930008091C6001F910F91FF90EF9008950E94D3
:10794000763C982F8091C00085FFFCCF9093C600B5
:1079500091362CF490330CF09053892F089597555D
:10796000892F08951F930E949F3C182F0E949F3CCF
:107970001295107F810F1F9108951F93182F882350
:1079800021F00E94763C1150E1F71F9108951F935A
:10799000182F0E94763C803249F0809103018F5F5E
:1079A000809303018530C1F01F9108958091C0003C
:1079B00085FFFCCF84E18093C6008091C00085FFE5
:1079C000FCCF1093C6008091C00085FFFCCF80E102
:1079D0008093C6001F910895E0910401F091050184
:1079E00009951F9108950E94763C803241F0809164
:1079F00003018F5F80930301853081F008958091AA
:107A0000C00085FFFCCF84E18093C6008091C00058
:107A100085FFFCCF80E18093C6000895E0910401CA
:107A2000F09105010995089540E951E08823A1F0FE
:107A30002D9A28EE33E0FA013197F1F721503040CA
:107A4000D1F72D9828EE33E0FA013197F1F7215064
:107A50003040D1F7815061F708953F924F925F9285
:107A60006F927F928F929F92AF92BF92CF92DF924E
:107A7000EF92FF920F931F93CF93DF93000080E16B
:107A80008093C4001092C50088E18093C10086E015
:107A90008093C2005098589A259A81E00E94143D24
:107AA00024E1F22E9EE1E92E85E9D82E0FE0C02ECA
:107AB00010E1B12EAA24A394B1E49B2EA6E58A2E50
:107AC000F2E57F2EE0E26E2E79E4572E63E5462E36
:107AD00050E5352E0E94763C8033B1F18133B9F107
:107AE000803409F46FC0813409F476C0823409F41B
:107AF00085C0853409F488C0803531F1823521F1A3
:107B0000813511F1853509F485C0863509F48DC0BC
:107B1000843609F496C0843709F403C1853709F423
:107B200072C1863709F466C0809103018F5F80932C
:107B30000301853079F6E0910401F0910501099582
:107B40000E94763C803351F60E94F33CC3CF0E94E2
:107B5000763C803249F78091C00085FFFCCFF092DF
:107B6000C6008091C00085FFFCCF9092C600809136
:107B7000C00085FFFCCF8092C6008091C00085FFC9
:107B8000FCCF7092C6008091C00085FFFCCF609250
:107B9000C6008091C00085FFFCCF5092C600809146
:107BA000C00085FFFCCF4092C6008091C00085FFD9
:107BB000FCCF3092C6008091C00085FFFCCFB09210
:107BC000C60088CF0E94763C863808F4BDCF0E945C
:107BD000763C0E94F33C7ECF0E94763C803809F4CC
:107BE0009CC0813809F40BC1823809F43CC1883942
:107BF00009F48FC080E00E94C73C6CCF84E10E94F2
:107C0000BD3C0E94F33C66CF85E00E94BD3C0E94D3
:107C1000F33C60CF0E94763C809306010E94763C44
:107C2000809307010E94F33C55CF0E94763C80333D
:107C300009F41DC183E00E94BD3C80E00E94C73C66
:107C400049CF0E94763C809309020E94763C809343
:107C5000080280910C028E7F80930C020E94763C79
:107C6000853409F415C18091080290910902892B8D
:107C700089F000E010E00E94763CF801E85FFE4FDA
:107C800080830F5F1F4F80910802909109020817AF
:107C9000190788F30E94763C803209F045CF809125
:107CA0000C0280FF01C16091060170910701660F0F
:107CB000771F7093070160930601A0910802B091AD
:107CC00009021097C9F0E8E0F1E09B01AD014E0F09
:107CD0005F1FF999FECF32BD21BD819180BDFA9A17
:107CE000F99A2F5F3F4FE417F50799F76A0F7B1F4B
:107CF00070930701609306018091C00085FFFCCF5F
:107D0000F092C6008091C00085FFFCCFB092C60003
:107D1000E1CE83E00E94C73CDDCE82E00E94C73CFA
:107D2000D9CE0E94763C809309020E94763C8093D3
:107D300008028091060190910701880F991F909386
:107D40000701809306010E94763C853409F4A6C0A1
:107D500080910C028E7F80930C020E94763C8032D0
:107D600009F0B8CE8091C00085FFFCCFF092C6002C
:107D7000609108027091090261157105B9F140E046
:107D800050E080910C02A82FA170B82FB27011C0E2
:107D9000BB2309F45CC0E0910601F0910701319624
:107DA000F0930701E09306014F5F5F4F46175707B7
:107DB000E8F4AA2369F3F999FECF209106013091E6
:107DC000070132BD21BDF89A90B58091C00085FFB2
:107DD000FCCF9093C6002F5F3F4F30930701209355
:107DE00006014F5F5F4F4617570718F38091C00099
:107DF00085FDE5CE8091C00085FFF8CFE0CE81E023
:107E00000E94C73C67CE0E94763C803209F08CCE3F
:107E10008091C00085FFFCCFF092C6008091C00029
:107E200085FFFCCFE092C6008091C00085FFFCCFAB
:107E3000D092C6008091C00085FFFCCFC092C600E2
:107E40008091C00085FFFCCFB092C60043CEE09188
:107E50000601F091070194918091C00085FFFCCF4D
:107E60009093C6009CCF80E10E94C73C33CE0E9415
:107E7000763C0E94763C182F0E94763C112309F430
:107E800083C0113009F484C08FE00E94C73C22CE29
:107E900080910C02816080930C02E5CE80910C02EF
:107EA000816080930C0259CF809107018823880F4D
:107EB000880B8A2180930B02809106019091070123
:107EC000880F991F90930701809306018091080203
:107ED00080FF09C080910802909109020196909359
:107EE000090280930802F894F999FECF1127E091D6
:107EF0000601F0910701C8E0D1E08091080290915D
:107F00000902103091F40091570001700130D9F34B
:107F100003E000935700E89500915700017001308D
:107F2000D9F301E100935700E89509901990009169
:107F3000570001700130D9F301E000935700E89534
:107F40001395103498F011270091570001700130FB
:107F5000D9F305E000935700E895009157000170B0
:107F60000130D9F301E100935700E895329602976A
:107F700009F0C7CF103011F00296E5CF112480919F
:107F8000C00085FFB9CEBCCE8EE10E94C73CA2CD19
:0C7F900085E90E94C73C9ECDF894FFCF0D
:027F9C00800063
:040000030000780081
:00000001FF
